:020000040000FA
:10000000AFEF01F0FFFFFFFF0EEF00F0FFFFFFFF7C
:10001000FFFFFFFFFFFFFFFF25EF00F081AC829C99
:1000200081AC22EF00F0828CD650F00ED714D8A409
:1000300000EE80F0D59ED6CFEEFFD7CFEEFFD76A89
:10004000D66AD58E8152F29011001000080E616FB1
:1000500062AF829A62BF828A0000808A809A623789
:10006000612F28EF00F01200948A080E616F626B16
:10007000D890623782BA6281808A809A612F39EF84
:1000800000F0949A1200080E686F10EE82F020EED5
:1000900070F0F29EE6CFDEFFE6CFDEFFF28E682F35
:1000A00049EF00F08098050E626F26EC00F06FB10A
:1000B000AA0E6FA1550E626F26EC00F069C062F0C7
:1000C00026EC00F06AC062F026EC00F06BC062F033
:1000D00026EC00F06CC062F026EC00F070C062F01C
:1000E00026EC00F071C062F026EC00F072C062F005
:1000F00026EC00F073C062F026EC00F074C062F0F1
:1001000026EC00F075C062F026EC00F076C062F0DC
:1001100026EC00F077C062F026EC00F078C062F0C8
:1001200026EC00F079C062F026EC00F07AC062F0B4
:1001300026EC00F07BC062F026EC00F07CC062F0A0
:1001400026EC00F07DC062F026EC00F07EC062F08C
:1001500026EC00F07FC062F026EC00F080881200F0
:100160008098000E626F26EC00F0000E626F26ECA5
:1001700000F080888098060E626F26EC00F0540E26
:10018000626F26EC00F0750E626F26EC00F0C50E73
:10019000626F26EC00F02A0E626F26EC00F0808879
:1001A0008098A00E626F26EC00F08088040EF76E37
:1001B000540EF66EFF0E636F330E606F632B0900F3
:1001C000F528FCE0809863C062F026EC00F0F5CFE3
:1001D00062F026EC00F08088602FDEEF00F080985F
:1001E000020E626F26EC00F0010E626F26EC00F04A
:1001F00080888098020E626F628D26EC00F000000D
:1002000034EC00F0808862B1F9EF00F08098240EA1
:10021000626F26EC00F0130E626F26EC00F080880F
:100220008098260E626F26EC00F03B0E626F26EC83
:1002300000F0808880980F0E626F26EC00F0000EB0
:10024000626F26EC00F080888098020E626F26ECC8
:1002500000F0020E626F26EC00F080888098020E9B
:10026000626F628D26EC00F0000034EC00F08088B4
:1002700062B32EEF01F080980F0E626F26EC00F053
:10028000A00E626F26EC00F080888098020E626FEC
:1002900026EC00F0020E626F26EC00F08088809859
:1002A000020E626F628D26EC00F0000034EC00F06C
:1002B000808862B34FEF01F08098250E626F26ECC4
:1002C00000F0080E626F26EC00F080881200676B69
:1002D0006F818098A00E626F26EC00F08088809875
:1002E000E00E626F26EC00F0808880980F0E626F3F
:1002F00026EC00F0010E626F26EC00F0808843ECE3
:1003000000F08098D00E626F26EC00F08088B190EB
:10031000270EB36EB31E100EB26EB21EA192B18044
:10032000A1A290EF01F067B7829C67A7828C672F2C
:1003300069EF01F012006D2FA8EF01F0100E6D6F44
:10034000040EF76E880EF66E6E51F626D8B0F72AB8
:100350000900F5CF66F069390F0B665F1200D38C88
:10036000D38AD388D3A4B2EF01F0806A816A826A0B
:10037000828C949C80889298828A949A809A929A8D
:100380007E6A7F6AD56AD580F294480ECB6ECA6ABF
:10039000CA8ACA829E92B16AB18EB18AA192DC0EDB
:1003A000826F846F866F886F8A6F8C6F8E6F906F8D
:1003B000050E836F856F876F896F8B6F8D6F8F6F62
:1003C000916FB190270EB36EB31E100EB26EB21EB7
:1003D000A192B180A1A2EAEF01F0B0EC00F0060E0C
:1003E000696F000E6A6F000E6B6F300E6C6F67ECFA
:1003F00001F06F6B6939F00B6E6F010E6D6FF28655
:100400007A8CD58EF28ECA849EA204EF02F09E9260
:100410008098A00E626F26EC00F080888098E00E35
:10042000626F26EC00F080889BEC01F080980F0E44
:10043000626F26EC00F066C062F026EC00F0808867
:1004400043EC00F08098D00E626F26EC00F08088BC
:1004500004EF02F0FF42001400FFFF000000000163
:10046000210500509E4B0002162B12006280800076
:100470000A32C30F13C300FF00003B00174780037D
:1004800001451800010FFF000A5A14641E6E2878F7
:1004900032823C8C469650A0A05096468C3C8232CC
:1004A00078286E1E64145A0A0A5A50A0146446969C
:1004B0001E6E3C8C28783282823278288C3C6E1EEC
:1004C00096466414A0505A0A28780A5A50A0146418
:1004D0001E6E3C8C32824696964682328C3C6E1E54
:1004E0006414A0505A0A782850A028780A5A1E6E20
:1004F0003C8C3282469614646414964682328C3C5C
:100500006E1E5A0A7828A05050A046963C8C287837
:100510000A5A32821E6E146464146E1E82325A0AA3
:1005200078288C3C9646A05046963C8C50A0287863
:100530000A5A1E6E32821464641482326E1E5A0A83
:100540007828A0508C3C964646960A5A3C8C1464F7
:1005500050A028781E6E328282326E1E7828A050FB
:1005600064148C3C5A0A964646960A5A50A03C8C13
:1005700028781E6E32821464641482326E1E7828CB
:100580008C3CA0505A0A9646FFFFFFFFFFFFFFFF7B
:10059000FFFFFFFFFFFFFFFFFFFFFFFFFFFFFFFF6B
:1005A000FFFFFFFFFFFFFFFFFFFFFFFFFFFFFFFF5B
:1005B000FFFFFFFFFFFFFFFFFFFFFFFFFFFFFFFF4B
:1005C000FFFFFFFFFFFFFFFFFFFFFFFFFFFFFFFF3B
:0200000400F00A
:100000004D434850FFFFFFFFFFFFFFFFFFFFFFFFD4
:10001000FFFFFFFFFFFFFFFFFFFFFFFFFFFFFFFFF0
:10002000FFFFFFFFFFFFFFFFFFFFFFFFFFFFFFFFE0
:10003000FFFFFFFFFFFFFFFFFFFFFFFFFFFFFFFFD0
:10004000FFFFFFFFFFFFFFFFFFFFFFFFFFFFFFFFC0
:10005000FFFFFFFFFFFFFFFFFFFFFFFFFFFFFFFFB0
:10006000FFFFFFFFFFFFFFFFFFFFFFFFFFFFFFFFA0
:10007000FFFFFFFFFFFFFFFFFFFFFFFFFFFFFFFF90
:10008000FFFFFFFFFFFFFFFFFFFFFFFFFFFFFFFF80
:10009000FFFFFFFFFFFFFFFFFFFFFFFFFFFFFFFF70
:1000A000FFFFFFFFFFFFFFFFFFFFFFFFFFFFFFFF60
:1000B000FFFFFFFFFFFFFFFFFFFFFFFFFFFFFFFF50
:1000C000FFFFFFFFFFFFFFFFFFFFFFFFFFFFFFFF40
:1000D000FFFFFFFFFFFFFFFFFFFFFFFFFFFFFFFF30
:1000E000FFFFFFFFFFFFFFFFFFFFFFFFFFFFFFFF20
:1000F000FFFFFFFFFFFFFFFFFFFFFFFFFFFFFFFF10
:020000040030CA
:0E000000000809140080800003C003E00340E4
:020000040020DA
:08000000FFFFFFFFFFFFFFFF00
:00000001FF
